BL51 BANKED LINKER/LOCATER V6.22                                                        02/28/2017  15:28:49  PAGE 1


BL51 BANKED LINKER/LOCATER V6.22, INVOKED BY:
E:\KEIL-C51\C51\BIN\BL51.EXE ..\OBJ\main.obj, ..\OBJ\LCD drive.obj TO ..\OBJ\13 PRINT (.\13.m51) RAMSIZE (256)


MEMORY MODEL: COMPACT


INPUT MODULES INCLUDED:
  ..\OBJ\main.obj (MAIN)
  ..\OBJ\LCD drive.obj (LCD_DRIVE)
  E:\KEIL-C51\C51\LIB\C51C.LIB (?C_STARTUP)


LINK MAP OF MODULE:  ..\OBJ\13 (MAIN)


            TYPE    BASE      LENGTH    RELOCATION   SEGMENT NAME
            -----------------------------------------------------

            * * * * * * *   D A T A   M E M O R Y   * * * * * * *
            REG     0000H     0008H     ABSOLUTE     "REG BANK 0"
            IDATA   0008H     0001H     UNIT         ?STACK

            * * * * * * *  X D A T A   M E M O R Y  * * * * * * *
            XDATA   0000H     001CH     INPAGE       _PDATA_GROUP_

            * * * * * * *   C O D E   M E M O R Y   * * * * * * *
            CODE    0000H     0003H     ABSOLUTE     
            CODE    0003H     0600H     UNIT         ?CO?LCD_DRIVE
            CODE    0603H     0275H     UNIT         ?PR?LCD_INIT?LCD_DRIVE
            CODE    0878H     00ECH     UNIT         ?PR?_GUI_SPRINTF_CHAR?LCD_DRIVE
            CODE    0964H     0064H     UNIT         ?PR?_GUI_SPRINTF_STRING?LCD_DRIVE
            CODE    09C8H     004CH     UNIT         ?PR?_LCD_TEST_SINGLECOLOR?LCD_DRIVE
            CODE    0A14H     0040H     UNIT         ?PR?_LCD_SETWINDOW?LCD_DRIVE
            CODE    0A54H     0036H     UNIT         ?PR?DISPLAY_ID?LCD_DRIVE
            CODE    0A8AH     0035H     UNIT         ?PR?MAIN?MAIN
            CODE    0ABFH     0027H     UNIT         ?PR?_GUI_POINT?LCD_DRIVE
            CODE    0AE6H     0025H     UNIT         ?PR?_DELAYMS?LCD_DRIVE
            CODE    0B0BH     001BH     UNIT         ?PR?HD_RESET?LCD_DRIVE
            CODE    0B26H     0014H     UNIT         ?PR?_LLCD_WRITE_DATA?LCD_DRIVE
            CODE    0B3AH     0014H     UNIT         ?PR?_LCD_SETXY?LCD_DRIVE
            CODE    0B4EH     0011H     UNIT         ?PR?_LLCD_WRITE_CMD?LCD_DRIVE
            CODE    0B5FH     000CH     UNIT         ?PR?_DELAYUS?LCD_DRIVE
            CODE    0B6BH     000CH     UNIT         ?C_C51STARTUP



OVERLAY MAP OF MODULE:   ..\OBJ\13 (MAIN)


SEGMENT                                       PDATA_GROUP
  +--> CALLED SEGMENT                       START    LENGTH
-----------------------------------------------------------
?C_C51STARTUP                               -----    -----
  +--> ?PR?MAIN?MAIN

?PR?MAIN?MAIN                               -----    -----
  +--> ?PR?HD_RESET?LCD_DRIVE
BL51 BANKED LINKER/LOCATER V6.22                                                      02/28/2017  15:28:49  PAGE 2


  +--> ?PR?LCD_INIT?LCD_DRIVE
  +--> ?PR?_DELAYMS?LCD_DRIVE
  +--> ?PR?_LCD_TEST_SINGLECOLOR?LCD_DRIVE
  +--> ?PR?DISPLAY_ID?LCD_DRIVE

?PR?HD_RESET?LCD_DRIVE                      -----    -----
  +--> ?PR?_DELAYMS?LCD_DRIVE

?PR?_DELAYMS?LCD_DRIVE                      0000H    0002H
  +--> ?PR?_DELAYUS?LCD_DRIVE

?PR?LCD_INIT?LCD_DRIVE                      -----    -----
  +--> ?PR?_LLCD_WRITE_CMD?LCD_DRIVE
  +--> ?PR?_LLCD_WRITE_DATA?LCD_DRIVE
  +--> ?PR?_DELAYMS?LCD_DRIVE
  +--> ?PR?_LCD_TEST_SINGLECOLOR?LCD_DRIVE

?PR?_LCD_TEST_SINGLECOLOR?LCD_DRIVE         0000H    0002H
  +--> ?PR?_LCD_SETWINDOW?LCD_DRIVE

?PR?_LCD_SETWINDOW?LCD_DRIVE                0016H    0006H
  +--> ?PR?_LLCD_WRITE_CMD?LCD_DRIVE
  +--> ?PR?_LLCD_WRITE_DATA?LCD_DRIVE

?PR?DISPLAY_ID?LCD_DRIVE                    -----    -----
  +--> ?CO?LCD_DRIVE
  +--> ?PR?_GUI_SPRINTF_STRING?LCD_DRIVE

?PR?_GUI_SPRINTF_STRING?LCD_DRIVE           0000H    0009H
  +--> ?PR?_GUI_SPRINTF_CHAR?LCD_DRIVE

?PR?_GUI_SPRINTF_CHAR?LCD_DRIVE             0009H    000BH
  +--> ?CO?LCD_DRIVE
  +--> ?PR?_GUI_POINT?LCD_DRIVE

?PR?_GUI_POINT?LCD_DRIVE                    0014H    0002H
  +--> ?PR?_LCD_SETXY?LCD_DRIVE

?PR?_LCD_SETXY?LCD_DRIVE                    -----    -----
  +--> ?PR?_LCD_SETWINDOW?LCD_DRIVE



SYMBOL TABLE OF MODULE:  ..\OBJ\13 (MAIN)

  VALUE           TYPE          NAME
  ----------------------------------

  -------         MODULE        MAIN
  C:0000H         SYMBOL        _ICE_DUMMY_
  D:0090H         PUBLIC        P1
  D:00B0H         PUBLIC        P3
  D:00A8H         PUBLIC        IE
  D:00B8H         PUBLIC        IP
  C:0A8AH         PUBLIC        main
  D:0098H         PUBLIC        SCON
  D:0088H         PUBLIC        TCON
BL51 BANKED LINKER/LOCATER V6.22                                                      02/28/2017  15:28:49  PAGE 3


  D:00C8H         PUBLIC        T2CON
  D:00D0H         PUBLIC        PSW
  -------         PROC          MAIN
  C:0A8AH         LINE#         3
  C:0A8AH         LINE#         4
  C:0A8AH         LINE#         6
  C:0A8DH         LINE#         7
  C:0A90H         LINE#         8
  C:0A90H         LINE#         9
  C:0A90H         LINE#         11
  C:0A9EH         LINE#         12
  C:0AA5H         LINE#         13
  C:0AB3H         LINE#         14
  C:0ABAH         LINE#         15
  C:0ABDH         LINE#         16
  -------         ENDPROC       MAIN
  -------         ENDMOD        MAIN

  -------         MODULE        LCD_DRIVE
  C:0000H         SYMBOL        _ICE_DUMMY_
  D:0090H         PUBLIC        P1
  D:00A0H         PUBLIC        P2
  D:00B0H         PUBLIC        P3
  C:0B29H         PUBLIC        _LLCD_WRITE_DATA
  D:00A8H         PUBLIC        IE
  C:0B0BH         PUBLIC        HD_reset
  D:00B8H         PUBLIC        IP
  C:0A14H         PUBLIC        _LCD_setwindow
  B:0090H.1       PUBLIC        RS
  D:0098H         PUBLIC        SCON
  D:0088H         PUBLIC        TCON
  C:09C8H         PUBLIC        _LCD_TEST_SingleColor
  C:0B4EH         PUBLIC        _LLCD_WRITE_CMD
  C:0A54H         PUBLIC        Display_ID
  C:0964H         PUBLIC        _GUI_sprintf_string
  C:0013H         PUBLIC        font16x8
  C:0878H         PUBLIC        _GUI_sprintf_char
  C:0ABFH         PUBLIC        _GUI_Point
  B:0090H.3       PUBLIC        RDB
  B:0090H.0       PUBLIC        TFT_CS
  D:00C8H         PUBLIC        T2CON
  C:0603H         PUBLIC        LCD_init
  B:0090H.4       PUBLIC        RES
  B:0090H.2       PUBLIC        WRB
  C:0AE6H         PUBLIC        _delayms
  C:0B3AH         PUBLIC        _LCD_setxy
  D:00D0H         PUBLIC        PSW
  C:0B5FH         PUBLIC        _delayus
  -------         PROC          DISPLAY_ID
  C:0A54H         LINE#         10
  C:0A54H         LINE#         11
  C:0A54H         LINE#         13
  C:0A6FH         LINE#         14
  -------         ENDPROC       DISPLAY_ID
  -------         PROC          LCD_INIT
  C:0603H         LINE#         21
  C:0603H         LINE#         22
BL51 BANKED LINKER/LOCATER V6.22                                                      02/28/2017  15:28:49  PAGE 4


  C:0603H         LINE#         23
  C:060AH         LINE#         24
  C:060DH         LINE#         25
  C:0614H         LINE#         26
  C:061BH         LINE#         27
  C:0622H         LINE#         28
  C:0629H         LINE#         29
  C:0630H         LINE#         30
  C:0637H         LINE#         31
  C:063EH         LINE#         32
  C:0645H         LINE#         33
  C:064CH         LINE#         34
  C:0653H         LINE#         35
  C:065AH         LINE#         36
  C:0661H         LINE#         37
  C:0668H         LINE#         38
  C:066FH         LINE#         39
  C:0672H         LINE#         40
  C:0679H         LINE#         41
  C:0680H         LINE#         42
  C:0687H         LINE#         43
  C:068EH         LINE#         44
  C:0695H         LINE#         45
  C:069BH         LINE#         46
  C:06A1H         LINE#         47
  C:06A8H         LINE#         48
  C:06AFH         LINE#         49
  C:06B6H         LINE#         50
  C:06BDH         LINE#         51
  C:06C4H         LINE#         52
  C:06CBH         LINE#         53
  C:06D2H         LINE#         54
  C:06D9H         LINE#         55
  C:06E0H         LINE#         56
  C:06E7H         LINE#         57
  C:06EEH         LINE#         58
  C:06F5H         LINE#         59
  C:06FCH         LINE#         60
  C:0703H         LINE#         61
  C:0709H         LINE#         62
  C:0710H         LINE#         63
  C:0717H         LINE#         64
  C:071EH         LINE#         65
  C:0725H         LINE#         66
  C:072CH         LINE#         67
  C:0732H         LINE#         68
  C:0739H         LINE#         69
  C:0740H         LINE#         70
  C:0747H         LINE#         71
  C:074EH         LINE#         72
  C:0755H         LINE#         73
  C:075CH         LINE#         74
  C:0763H         LINE#         75
  C:076AH         LINE#         76
  C:0771H         LINE#         77
  C:0778H         LINE#         78
  C:077FH         LINE#         79
BL51 BANKED LINKER/LOCATER V6.22                                                      02/28/2017  15:28:49  PAGE 5


  C:0786H         LINE#         80
  C:078DH         LINE#         81
  C:0794H         LINE#         82
  C:079AH         LINE#         83
  C:07A0H         LINE#         84
  C:07A6H         LINE#         85
  C:07ACH         LINE#         86
  C:07B3H         LINE#         87
  C:07B9H         LINE#         88
  C:07C0H         LINE#         89
  C:07C7H         LINE#         90
  C:07CEH         LINE#         91
  C:07D5H         LINE#         92
  C:07DCH         LINE#         93
  C:07E3H         LINE#         94
  C:07EAH         LINE#         95
  C:07F1H         LINE#         96
  C:07F8H         LINE#         97
  C:07FFH         LINE#         98
  C:0806H         LINE#         99
  C:080DH         LINE#         100
  C:0814H         LINE#         101
  C:081BH         LINE#         102
  C:0822H         LINE#         103
  C:0828H         LINE#         104
  C:082EH         LINE#         105
  C:0835H         LINE#         106
  C:083CH         LINE#         107
  C:0843H         LINE#         108
  C:0849H         LINE#         109
  C:084FH         LINE#         110
  C:0855H         LINE#         111
  C:085CH         LINE#         116
  C:0863H         LINE#         117
  C:086AH         LINE#         118
  C:0871H         LINE#         119
  -------         ENDPROC       LCD_INIT
  -------         PROC          HD_RESET
  C:0B0BH         LINE#         127
  C:0B0BH         LINE#         128
  C:0B0BH         LINE#         129
  C:0B0DH         LINE#         130
  C:0B14H         LINE#         131
  C:0B16H         LINE#         132
  C:0B1DH         LINE#         133
  C:0B1FH         LINE#         134
  -------         ENDPROC       HD_RESET
  -------         PROC          _LLCD_WRITE_CMD
  D:0006H         SYMBOL        cmd
  C:0B4EH         LINE#         141
  C:0B4EH         LINE#         142
  C:0B4EH         LINE#         144
  C:0B50H         LINE#         145
  C:0B52H         LINE#         146
  C:0B54H         LINE#         147
  C:0B56H         LINE#         148
  C:0B58H         LINE#         149
BL51 BANKED LINKER/LOCATER V6.22                                                      02/28/2017  15:28:49  PAGE 6


  C:0B5AH         LINE#         150
  C:0B5CH         LINE#         151
  C:0B5EH         LINE#         153
  -------         ENDPROC       _LLCD_WRITE_CMD
  -------         PROC          L?0045
  -------         ENDPROC       L?0045
  -------         PROC          _LLCD_WRITE_DATA
  D:0006H         SYMBOL        dataa
  C:0B29H         LINE#         158
  C:0B29H         LINE#         159
  C:0B29H         LINE#         161
  C:0B2BH         LINE#         162
  C:0B2DH         LINE#         163
  C:0B2FH         LINE#         164
  C:0B31H         LINE#         166
  C:0B33H         LINE#         167
  C:0B35H         LINE#         168
  C:0B37H         LINE#         169
  C:0B39H         LINE#         171
  -------         ENDPROC       _LLCD_WRITE_DATA
  -------         PROC          _GUI_SPRINTF_STRING
  X:0000H         SYMBOL        x
  X:0001H         SYMBOL        y
  X:0003H         SYMBOL        s
  X:0005H         SYMBOL        color
  X:0007H         SYMBOL        b_color
  C:0964H         LINE#         177
  C:0974H         LINE#         178
  C:0974H         LINE#         179
  C:0983H         LINE#         180
  C:0983H         LINE#         181
  C:09B4H         LINE#         182
  C:09BAH         LINE#         183
  C:09C7H         LINE#         186
  -------         ENDPROC       _GUI_SPRINTF_STRING
  -------         PROC          _GUI_SPRINTF_CHAR
  X:0009H         SYMBOL        x
  X:000AH         SYMBOL        y
  X:000CH         SYMBOL        c
  X:000DH         SYMBOL        color
  X:000FH         SYMBOL        b_color
  -------         DO            
  X:0011H         SYMBOL        s_x
  X:0012H         SYMBOL        s_y
  X:0013H         SYMBOL        temp
  D:0006H         SYMBOL        j
  -------         ENDDO         
  C:0878H         LINE#         191
  C:0885H         LINE#         192
  C:0885H         LINE#         195
  C:0889H         LINE#         196
  C:0899H         LINE#         197
  C:0899H         LINE#         198
  C:08B2H         LINE#         199
  C:08B2H         LINE#         200
  C:08B7H         LINE#         201
  C:08CAH         LINE#         202
BL51 BANKED LINKER/LOCATER V6.22                                                      02/28/2017  15:28:49  PAGE 7


  C:08D9H         LINE#         204
  C:08E6H         LINE#         205
  C:08E6H         LINE#         206
  C:08FAH         LINE#         207
  C:08FAH         LINE#         208
  C:091FH         LINE#         209
  C:091FH         LINE#         210
  C:0931H         LINE#         211
  C:0933H         LINE#         213
  C:0933H         LINE#         214
  C:0954H         LINE#         215
  C:0954H         LINE#         216
  C:0954H         LINE#         217
  C:095BH         LINE#         218
  C:095BH         LINE#         219
  C:0963H         LINE#         220
  -------         ENDPROC       _GUI_SPRINTF_CHAR
  -------         PROC          _GUI_POINT
  D:0007H         SYMBOL        x
  D:0004H         SYMBOL        y
  X:0014H         SYMBOL        color
  C:0ABFH         LINE#         225
  C:0AC6H         LINE#         226
  C:0AC6H         LINE#         227
  C:0AC9H         LINE#         228
  C:0ACBH         LINE#         229
  C:0ACDH         LINE#         230
  C:0ACFH         LINE#         231
  C:0AD9H         LINE#         232
  C:0ADBH         LINE#         233
  C:0ADDH         LINE#         235
  C:0ADFH         LINE#         236
  C:0AE1H         LINE#         237
  C:0AE3H         LINE#         238
  C:0AE5H         LINE#         239
  -------         ENDPROC       _GUI_POINT
  -------         PROC          _LCD_SETXY
  D:0006H         SYMBOL        x
  D:0082H         SYMBOL        y
  C:0B3AH         LINE#         244
  C:0B40H         LINE#         245
  C:0B40H         LINE#         246
  -------         ENDPROC       _LCD_SETXY
  -------         PROC          _LCD_SETWINDOW
  D:0002H         SYMBOL        x0
  D:0004H         SYMBOL        y0
  D:0003H         SYMBOL        x1
  X:001AH         SYMBOL        y1
  C:0A14H         LINE#         252
  C:0A16H         LINE#         253
  C:0A16H         LINE#         254
  C:0A1DH         LINE#         255
  C:0A22H         LINE#         256
  C:0A27H         LINE#         257
  C:0A2CH         LINE#         258
  C:0A31H         LINE#         260
  C:0A36H         LINE#         261
BL51 BANKED LINKER/LOCATER V6.22                                                      02/28/2017  15:28:49  PAGE 8


  C:0A3BH         LINE#         262
  C:0A42H         LINE#         263
  C:0A49H         LINE#         264
  C:0A4FH         LINE#         266
  -------         ENDPROC       _LCD_SETWINDOW
  -------         PROC          _LCD_TEST_SINGLECOLOR
  X:0000H         SYMBOL        color
  -------         DO            
  D:0004H         SYMBOL        i
  D:0002H         SYMBOL        j
  -------         ENDDO         
  C:09C8H         LINE#         272
  C:09CFH         LINE#         273
  C:09CFH         LINE#         276
  C:09E1H         LINE#         278
  C:09E3H         LINE#         279
  C:09E5H         LINE#         280
  C:09E7H         LINE#         282
  C:09E7H         LINE#         283
  C:09E7H         LINE#         284
  C:09EAH         LINE#         285
  C:09EAH         LINE#         286
  C:09EFH         LINE#         287
  C:09F1H         LINE#         288
  C:09F3H         LINE#         290
  C:09F7H         LINE#         291
  C:09F9H         LINE#         292
  C:09FBH         LINE#         293
  C:0A06H         LINE#         294
  C:0A11H         LINE#         296
  C:0A13H         LINE#         297
  -------         ENDPROC       _LCD_TEST_SINGLECOLOR
  -------         PROC          _DELAYMS
  X:0000H         SYMBOL        value
  C:0AE6H         LINE#         303
  C:0AEDH         LINE#         304
  C:0AEDH         LINE#         305
  C:0AF6H         LINE#         306
  C:0AF6H         LINE#         307
  C:0AFDH         LINE#         308
  C:0B08H         LINE#         309
  C:0B0AH         LINE#         310
  -------         ENDPROC       _DELAYMS
  -------         PROC          _DELAYUS
  D:0006H         SYMBOL        value1
  C:0B5FH         LINE#         315
  C:0B5FH         LINE#         316
  C:0B5FH         LINE#         317
  C:0B63H         LINE#         318
  C:0B6AH         LINE#         319
  -------         ENDPROC       _DELAYUS
  -------         ENDMOD        LCD_DRIVE

Program Size: data=9.0 xdata=28 code=2935
LINK/LOCATE RUN COMPLETE.  0 WARNING(S),  0 ERROR(S)
